:10000000C2EF12F0202020202020202020202020BD
:100010002020202000002D2D2D2D2D2D2D2D2D2D9E
:100020002D2D000025352E32664D204F686D0000C5
:1000300025362E32666B204F686D000025382E3233
:1000400066204F686D0020302E31200020203120A6
:1000500000002020203120002031302000002039F5
:100060002E3120002031302000002031303020009F
:10007000203130302000202020316B0020393130F9
:100080002000202020316B00202031306B002039EF
:100090002E316B00202031306B00202039316B0075
:1000A000203130306B00202020314D00203931309C
:1000B0006B00202020314D00202031304D002D2DAF
:1000C0002D2D2D0034373020200031306B202000C2
:1000D0003130306B2000314D202020005220202074
:1000E0000000453234200000202020200000EA6A71
:1000F000480EE96EEF500DE00A0E016E006A002E08
:10010000FED7012EFBD75F0E006E002EFED7EF2E1E
:10011000F3D7120093909392939493969398939A13
:1001200089969296929E898A929A8B8094808B88E7
:1001300094888B8A948A8B8C948C8B8E948E8B82F1
:1001400094828B8494848B869486C050C00B07095C
:10015000C06EC08EC2800F015C51800B5C6F010EBF
:100160005D6FC196C198C19A000E016EC250830B9B
:100170000110C26E000E016EC150F80B0110C16E6D
:10018000870ECD6EAA6A0001E6EF12F0899A5A6ACC
:100190005A500F0812E3000B006E5950800B036E8B
:1001A0000050031002E0898E01D0899E89868996CD
:1001B000D890583659365A2AEBD7898A12EF01F06F
:1001C0005450010A0FE0030A0FE0060A10E0010A8A
:1001D00011E00D0A12E0020A13E01A0A14E0300AD4
:1001E00015E018D0556A16D0010E556E13D0020EC8
:1001F000556E10D0030E556E0DD0040E556E0AD0FC
:10020000050E556E07D0060E556E04D0070E556EBE
:1002100001D0556A55C056F0400E576E596E55C004
:1002200058F0B4D7120066A902D08A8001D08A9013
:1002300066A702D08A8A01D08A9A66A502D08A88E7
:1002400001D08A9866A302D08A8601D08A9666A1D8
:1002500002D08A8401D08A9412008A8200D08A92C5
:1002600000D01200640E486E42DF030E666FDBDFC3
:10027000F4DF050E486E3BDF030E666FD4DFEDDF63
:10028000010E486E34DF030E666FCDDFE6DF010E30
:10029000486E2DDF020E666FC6DFDFDF010E486E8F
:1002A00026DF020E666FBFDFD8DF010E486E1FDF4C
:1002B0000E0E666FB8DFD1DF010E486E18DF666B79
:1002C000B2DFCBDF010E486E12DF080E666FABDFC8
:1002D000C4DF010E486E0BDF666BA5DFBEDF010ECB
:1002E000486E05DF0C0E666F9EDFB7DF010E486EAD
:1002F000FEDE666B98DFB1DF010E486EF8DE060E9B
:10030000666F91DFAADF010E486EF1DE666B8BDF50
:10031000A4DF010E486EEBDE010E666F84DF9DDF09
:10032000020E486EE4DEF0EF12F0666B7CDF95DFC4
:10033000020E666F78DF91DF020E486ED8DEF2EFB4
:1003400012F05450000A07E0010A0AE0030A0DE027
:10035000010A10E014D094909482948494860FD073
:1003600094929480948494860AD0949494809482F5
:10037000948605D0949694809482948400D0120040
:10038000C2825C90C2A25C805CB004D05C90C2A2CD
:100390005C80FAD7C2B2FED7C4CF03F0C3CF5DF002
:1003A000C4CF5EF05DC001F05EC002F0E4EF01F08A
:1003B000576A566A556A546A596A586A595211E11D
:1003C00058503F080EE3DCD702C003F0015054261A
:1003D00002505522000E56225722582AD8B4592AC4
:1003E000EDD7573256325532543257325632553293
:1003F00054325732563255325432573256325532C1
:1004000054325732563255325432573256325532B0
:100410005432030E571655C05BF054C05AF05AC000
:1004200001F05BC002F01200526A010E536E52508E
:100430000BE0010A0DE0030A0FE0010A11E0070AD0
:1004400013E0010A15E018D0010E546EB9DE14D085
:10045000020E546EB5DE10D0040E546EB1DE0CD018
:10046000080E546EADDE08D0100E546EA9DE04D016
:10047000200E546EA5DE00D0010E536E546A61DF6B
:100480001A0E006E002EFED7000092DF02C04BF065
:1004900001C04AF0010E546E54DF1A0E006E002E99
:1004A000FED7000085DF02C04DF001C04CF0020E07
:1004B000546E47DF1A0E006E002EFED7000078DF64
:1004C00002C04FF001C04EF0030E546E3ADF1A0E18
:1004D000006E002EFED700006BDF02C051F001C09D
:1004E00050F05250080DF350556A546E040E5424C7
:1004F000E96E000E5520EA6E4BC0ECFFED524AC08B
:10050000EFFF5250080DF350556A546E020E5424FA
:10051000016E000E5520036E0150040FE96E000EAF
:100520000320EA6E4DC0ECFFED524CC0EFFF52507D
:10053000080DF350556A546E040E5424016E000EDB
:100540005520036E0150040FE96E000E0320EA6E81
:100550004FC0ECFFED524EC0EFFF5250080DF3506C
:10056000556A546E060E5424016E000E5520036E1B
:100570000150040FE96E000E0320EA6E51C0ECFF3B
:10058000ED5250C0EFFF522A010E525C080DF3509D
:10059000556A546E040E5424E96E000E5520EA6E1E
:1005A000ECCF57F0ED52EFCF56F05750030808E369
:1005B00003E15650E70804E352500608D8A437D7A1
:1005C000520652C036F0376A5250080DF350556A41
:1005D000546E040E5424E96E000E5520EA6EECCFE2
:1005E00057F0ED52EFCF56F057500E0806E303E1F7
:1005F00056508A0802E3376A5FD05250080DF35014
:10060000556A546E020E5424016E000E5520036E7E
:100610000150040FE96E000E0320EA6EECCF55F096
:10062000ED52EFCF54F055500E0807E303E154505C
:100630008A0803E3010E376E3FD05250080DF35085
:10064000556A546E040E5424016E000E5520036E3C
:100650000150040FE96E000E0320EA6EECCF55F056
:10066000ED52EFCF54F055500E0807E303E154501C
:100670008A0803E3020E376E1FD05250080DF35064
:10068000556A546E060E5424016E000E5520036EFA
:100690000150040FE96E000E0320EA6EECCF55F016
:1006A000ED52EFCF54F055500E0806E303E15450DD
:1006B0008A0802E3030E376E3650080DF350556A70
:1006C000546ED8903734036A5424016E5550032277
:1006D0000150040FE96E000E0320EA6EECCF39F0F2
:1006E000ED52EFCF38F0F4EF12F08E0E006E55C0E1
:1006F00001F054C002F0036A015209E102C001F0A6
:10070000026A080E005E015202E1006A08D0D89029
:1007100001BE04D0023601360006F9D7019E68EF0B
:1007200006F06451D8B471D0006E6851D8B46DD061
:10073000002604E3810E002668E204D07F0E005EEE
:1007400064E363E065C06CF069516C1B658F698F71
:1007500067516B03F4CF6EF066516A03F4CF03F078
:10076000F3CF6DF06B03F3506E27F4506D23000E42
:10077000032267516A03F3506E27F4506D23000E75
:10078000026A0322022265516B03F3506D27F45075
:100790000322000E022265516A03F3500326F4502F
:1007A0000222000E016A012267516903F3506D278E
:1007B000F4500322000E0222012266516903F35015
:1007C0000326F4500222000E012265516903F35002
:1007D0000226F4500122002A01BE05D06D370336EF
:1007E000023601360006000E6DAF0AD0032A02223F
:1007F0000122015005E1025003E1035001E1002A0A
:100800006CBF018E6CAF019E04D0006A016A026A5F
:10081000036A1200800ED8B2691B6E6B6F6B65C0E5
:100820006DF069516D1B6451D8B4DCD06C6F006EF3
:100830006851D8B4E0D06C5FD8B481D03DE369C0D2
:1008400072F0728F6AC071F06BC070F06F6BD890ED
:100850007233713370336F336C2FF8D76DAF03D0B1
:100860006E81DDD06E916C916E89EA6A670EE96ED9
:10087000E9D06E996DBF0AD06CA113D07233713379
:1008800070336F33002AD8B4C5D00BD072BF0CD0F0
:10089000D8906F377037713772370006D8B4BAD036
:1008A000F5D76E8D6BD06E9D65C06DF065AF02D0D3
:1008B000728FA9D0729FA7D068C06CF068C000F09A
:1008C00064516C5F65C072F0728F66C071F067C072
:1008D00070F06F6BD8907233713370336F336C2F4D
:1008E000F8D76DAF03D06E839AD06E936C916E8BF8
:1008F000EA6A6B0EE96EA6D06E9B6DBF0AD06CA142
:1009000013D07233713370336F33002AD8B482D06E
:100910000BD072BF0CD0D8906F37703771377237E9
:100920000006D8B477D0F5D76E8F28D06E9F69C0F7
:100930006DF069AF02D0728F66D0729F64D069C0CB
:1009400072F0728F6AC071F06BC070F06DAF04D03E
:10095000729F6E8564D06E956F6B6C91EA6A670EBC
:10096000E96E70D06DBF1CD065C06DF06CA106D073
:100970007233713370336F33002A4CE06FAF0BD09A
:10098000702B09E1712B07E1722B05E17233713392
:100990007033002A3FE06EBD86D76EBFC7D71CD02C
:1009A000800E721B72AF04D03AD069C06DF00AD0CD
:1009B00065C06DF0725306E1715304E1705302E1BA
:1009C000006A21D072BF08D0D8906F377037713766
:1009D0007237002EF7D71ED06DAF02D0728F13D0B2
:1009E000729F11D068C000F069C072F06AC071F0E7
:1009F0006BC070F008D064C000F065C072F066C0D3
:100A000071F067C070F072C001F071C002F070C088
:100A100003F034D0006A016A026A036A2FD06F6B58
:100A2000701F711F721F6F1F6F2B05E1702B03E189
:100A3000712B01E1722B6EB115D76EB356D76EB51F
:100A40008AD7B3D7EF50702705E3712B03E1722BE0
:100A5000D8B46C81ED52EF50712703E3722BD8B4F8
:100A60006C81ED52EF50EFBE01D0800A7227D8B0F2
:100A70006C816EB9FED66EBB3FD774D7120058504A
:100A8000D8B4A5D0646F5C50D8B4A1D0645F05E33E
:100A90007F0E6427D8B09BD006D0810E645FD8A0AB
:100AA00096D0D8B494D064C000F0016A026A036A98
:100AB000636B59C062F0628F5AC061F05BC060F036
:100AC000190E646F5F50605F0DE2010E615F0AE214
:100AD000625F08E2635F06E2632B622B612B5F506B
:100AE000602728D05E50615F12E2010E625F0FE264
:100AF000635F0DE2632B622B5E5061275F506027BE
:100B000019E3612B17E1622B15E1632B13D05D50C4
:100B10008009625F0EE2010E635F0BE2632B5D50A2
:100B2000800962275E506127E9E3622BE7E1632BCE
:100B3000E5D70380642F01D00BD0D89060376137A0
:100B400062376337D8900336023601366537BAD735
:100B500065A106D0D890013202320332653302D04B
:100B6000000635E065BF1ED0D89060376137623728
:100B700063375F50605F07E2010E615F04E2625F0E
:100B800002E2635F1AE35E50615F05E2010E625F9D
:100B900002E2635F12E35D508009625F03E2010ECF
:100BA000635F0BE3032A09E1022A07E1012A05E159
:100BB000002A0DE001320232033259C064F05D5068
:100BC000641B64AF02D0018E06D0019E04D0006A7F
:100BD000016A026A036A12003750000A07E0010A3C
:100BE0000CE0030A12E0010A19E021D04B6A4A6ABC
:100BF000090E496E880E486E1AD04B6A640E4A6E12
:100C00001D0E496E8C0E486E12D0800E4B6E740E07
:100C10004A6E430E496E8F0E486E09D0900E4B6E91
:100C2000280E4A6E740E496E920E486E00D03650F1
:100C30000BE0010A0FE0030A13E0010A17E0070ABC
:100C40001BE0010A1FE024D04F6A4E6A4D6A7F0EF6
:100C50004C6E1ED04F6A4E6A4D6A800E4C6E18D094
:100C60004F6A4E6A4D6A810E4C6E12D04F6A4E6AC0
:100C70004D6A820E4C6E0CD04F6A4E6A4D6A830EDE
:100C80004C6E06D04F6A4E6A4D6A840E4C6E00D090
:100C900039500D080EE2FF0A03E138508B0809E2D3
:100CA000800E536E960E526E180E516E960E506E4A
:100CB00071D0395208E13850310805E3536A526A5D
:100CC000516A506A67D039C055F038C054F00DD51C
:100CD00003C053F002C052F001C051F000C050F008
:100CE00053C067F052C066F051C065F050C064F068
:100CF0004BC06BF04AC06AF049C069F048C068F068
:100D000010DD03C057F002C056F001C055F000C01E
:100D100054F0676B666B656B8B0E646F4FC06BF046
:100D20004EC06AF04DC069F04CC068F0FADC03C0F8
:100D30005BF002C05AF001C059F000C058F0D882F0
:100D400003C067F002C066F001C065F000C064F047
:100D500053C06BF052C06AF051C069F050C068F0E7
:100D600059DD57C05BF056C05AF055C059F054C019
:100D700058F003C05FF002C05EF001C05DF000C03B
:100D80005CF07DDE03C053F002C052F001C051F0B0
:100D900000C050F050C000F051C001F052C002F04D
:100DA00053C003F0F6EF12F04C38006E0F0E001631
:100DB00000500F0B4E6E4C500F0B4D6E4EC066F038
:100DC00013EC01F02DEC01F06A0E006E002EFED740
:100DD00000004DC066F013EC01F02DEC01F06A0E3E
:100DE000006E002EFED700000FEF07F04950000AFA
:100DF00007E0010A06E0030A07E0010A08E00AD05A
:100E000009D0400E482606D0140E482603D0540EB2
:100E1000482600D0800E48244B6E4C6EC5D7120079
:100E20006339646F0F0E64176317100E6425656FC6
:100E3000666F13EC01F02DEC01F0100E6325656F69
:100E4000666F13EC01F02DEC01F06A0E006E002EBF
:100E5000FED7000012000900F5520CE0F6CF52F068
:100E6000F7CF53F0F5CF63F0DBDF52C0F6FF53C08E
:100E7000F7FFF1D7120053C05AF057505A1A5AAE22
:100E800005D0D894D89053BED8802FD053C05AF0F4
:100E900056C05BF052505B5E06E05AAE26D0D8508A
:100EA000010AD86E22D057C05BF053505B5E06E05B
:100EB0005AAE1BD0D850010AD86E17D058C05BF07C
:100EC00054505B5E06E05AAE10D0D850010AD86E7E
:100ED0000CD059C05BF055505B5E06E05AAE05D0B1
:100EE000D850010AD86E01D0D89012006351B608CC
:100EF000636F036A64C067F0648FD89064336533AE
:100F000066330332023201320032632FF6D767AF05
:100F10000BD0001E011E021E031E002AD8B4012A97
:100F2000D8B4022AD8B4032A05EF08F0D8B203D007
:100F3000EA6A6B0EE96E006A016A026A036A6B6B09
:100F40006C6B6D6B6E6B6A516911681167112CE0E7
:100F5000200E6F6FD89063376437653766376B370D
:100F60006C376D376E376A516E5D08E169516D5DA2
:100F700005E168516C5D02E167516B5D0FE36751FC
:100F80006B5F6851D8A0683D6C5F6951D8A0693D1E
:100F90006D5F6A51D8A06A3D6E5FD8800036013619
:100FA000023603366F2FD6D76BC0EFFF6CC0ECFF55
:100FB0006DC0ECFF6EC0ECFF1200E9505B6E5A5042
:100FC0005D6E1AE059C067F058C066F057C065F012
:100FD00056C064F06B6B6A6B200E696F820E686F8F
:100FE00091EC03F003C059F002C058F001C057F073
:100FF00000C056F05D2EE6D759C066F058C065F0C7
:1010000057C064F056C063F071D703C059F002C0F6
:1010100058F001C057F000C056F059AE0DD05B0635
:101020005B8A561E571E581E591E562AD8B4572A78
:10103000D8B4582AD8B4592A3B0E626F9A0E616F01
:10104000CA0E606F5F6A0A0E5D6E5A50D8B45B2A92
:10105000D882EA6A560EE96E59C066F058C065F04B
:1010600057C064F056C063F062C06AF061C069F0B6
:1010700060C068F05FC067F059DF015000520FE1B7
:101080005A285D5C0CE05B500CE00F0B5D5C01E0EE
:1010900037E25BBE35D05BBC04D0200E2DD0200ED5
:1010A0005B165BAA0CD05B9A5A50D8A45B06005022
:1010B0005B6E2D0E636FB4DE5B50006E5B6A5A5040
:1010C0005D5C0AE100505B6E2E0E636FA9DE5B5023
:1010D000006E200E5B16000E300E5BAA0DD05B9AE0
:1010E0005A50D8A45B0600505B6E2D0E636F98DEDD
:1010F0005B50006E5B6A300E002600C063F090DE2D
:10110000D89262C066F061C065F060C064F05FC0F4
:1011100063F06A6B696B686B0A0E676F07DF03C069
:1011200062F002C061F001C060F000C05FF05D2EAF
:101130008FD712000900F6CF51F0F7CF52F0F5CF5C
:1011400063F06EDE51C0F6FF52C0F7FF502EF2D7AB
:101150001200600E556EF50E546E100E536E960E04
:10116000526E4BC059F04AC058F049C057F048C0C1
:1011700056F081DE06E3160EF66E000EF76E6BDE9D
:101180008FD0556AEF0E546E670E536E920E526EEC
:101190004BC059F04AC058F049C057F048C056F00B
:1011A0006ADE2DE34BC05BF04AC05AF049C059F0EB
:1011B00048C058F05F6A240E5E6E740E5D6E920E2B
:1011C0005C6E5DDC03C04FF002C04EF001C04DF01C
:1011D00000C04CF0040EE96E03C059F002C058F094
:1011E00001C057F000C056F0020E5A6EE6DE290E1E
:1011F000F66E000EF76E050E506E9CDF51D0556AEC
:10120000700E546E140E536E8C0E526E4BC059F00D
:101210004AC058F049C057F048C056F02CDE2CE3C5
:101220004BC05BF04AC05AF049C059F048C058F072
:101230005F6A5E6A7A0E5D6E880E5C6E20DC03C0AB
:101240004FF002C04EF001C04DF000C04CF0050E52
:10125000E96E03C059F002C058F001C057F000C059
:1012600056F0020E5A6EA9DE350EF66E000EF76EBF
:10127000050E506E5FDF14D0070EE96E4BC059F0BB
:101280004AC058F049C057F048C056F0020E5A6E96
:1012900094DE410EF66E000EF76E040E506E4ADFBD
:1012A00012EF13F08E0E006E6451005E65C002F006
:1012B00066C001F0028E005209E0D890025202E1AD
:1012C000015204E002320132002EF7D765AF05D09B
:1012D000011E021E012AD8B4022A120059C067F06A
:1012E00058C066F057C065F056C064F06B6B800E56
:1012F0006A6F3B0E696F8A0E686F91EC03F003C052
:1013000061F002C060F001C05FF000C05EF061C03B
:1013100067F060C066F05FC065F05EC064F0C2DF79
:1013200002C063F001C062F063510B080DE303E1FA
:1013300062512A0809E3C30E616FF50E606F680EF3
:101340005F6E7E0E5E6E2ED263510A0812E2FF0AB5
:1013500003E162512A080DE263510C080AE303E13C
:1013600062514E0806E3616B606B5F6A7F0E5E6ED2
:1013700019D263510B0815E2FF0A03E162514D08CF
:1013800010E263510D080DE303E162517A0809E3AD
:10139000CD0E616FCC0E606F0C0E5F6E7F0E5E6EB9
:1013A00001D263510C0815E2FF0A03E1625179088A
:1013B00010E263510E080DE303E16251A60809E350
:1013C0009A0E616F990E606F190E5F6E7F0E5E6EE2
:1013D000E9D163510D0814E2FF0A03E16251A50847
:1013E0000FE2635110080CE303E16251680808E35F
:1013F000660E616F606F260E5F6E7F0E5E6ED2D1DD
:1014000063510F0813E2FF0A03E1625167080EE21D
:10141000635112080BE303E162512A0807E3616B91
:10142000606B400E5F6E7F0E5E6EBCD16351110823
:1014300015E2FF0A03E16251290810E26351130823
:101440000DE303E16251EC0809E3CD0E616FCC0EB0
:10145000606F4C0E5F6E7F0E5E6EA4D163511208FA
:1014600013E2FF0A03E16251EB080EE26351160832
:101470000BE303E16251440807E3660E616F606F9E
:101480005F6E7F0E5E6E8ED16351150812E2FF0A09
:1014900003E1625143080DE2635118080AE303E1D6
:1014A00062519C0806E3616B606B5F6A800E5E6E42
:1014B00079D16351170815E2FF0A03E162519B08D5
:1014C00010E263511A080DE303E16251F40809E3E5
:1014D000CD0E616FCC0E606F0C0E5F6E800E5E6E77
:1014E00061D16351190815E2FF0A03E16251F30863
:1014F00010E263511D080DE303E16251E20809E3C4
:101500009A0E616F990E606F190E5F6E800E5E6E9F
:1015100049D163511C0815E2FF0A03E16251E10859
:1015200010E2635121080DE303E16251660809E30B
:10153000CD0E616FCC0E606F2C0E5F6E800E5E6EF6
:1015400031D16351200813E2FF0A03E162516508BB
:101550000EE2635124080BE303E16251EA0807E35A
:10156000616B606B400E5F6E800E5E6E1BD16351CF
:10157000230814E2FF0A03E16251E9080FE2635114
:1015800028080CE303E162516E0808E3330E616F33
:10159000606F530E5F6E800E5E6E04D1635127083C
:1015A00013E2FF0A03E162516D080EE263512B085A
:1015B0000BE303E16251F20807E3660E616F606FAF
:1015C0005F6E800E5E6EEED063512A0815E2FF0A50
:1015D00003E16251F10810E2635130080DE303E1C9
:1015E00062510C0809E39A0E616F990E606F790ED3
:1015F0005F6E800E5E6ED6D063512F0815E2FF0A33
:1016000003E162510B0810E2635134080DE303E17A
:101610006251BC0809E39A0E616F990E606F090E62
:101620005F6E810E5E6EBED06351330814E2FF0A16
:1016300003E16251BB080FE2635139080CE303E197
:1016400062516C0808E3660E616F606F160E5F6E84
:10165000810E5E6EA7D06351380814E2FF0A03E1E1
:1016600062516B080FE263513E080CE303E16251E3
:10167000B20808E3330E616F606F230E5F6E810E58
:101680005E6E90D063513D0813E2FF0A03E16251A0
:10169000B1080EE2635145080BE303E162512408EF
:1016A00007E3330E616F606F5F6E810E5E6E7AD0FE
:1016B0006351440814E2FF0A03E1625123080FE278
:1016C00063514C080CE303E162512C0808E3660EF9
:1016D000616F606F460E5F6E810E5E6E63D0635108
:1016E0004B0815E2FF0A03E162512B0810E2635137
:1016F00053080DE303E16251CA0809E39A0E616FD2
:10170000990E606F590E5F6E810E5E6E4BD0635105
:10171000520813E2FF0A03E16251C9080EE2635165
:101720005B080BE303E16251FE0807E3616B606B4A
:10173000700E5F6E810E5E6E35D063515A0814E2F2
:10174000FF0A03E16251FD080FE2635165080CE3F3
:1017500003E162515E0808E3330E616F606F030EB0
:101760005F6E820E5E6E1ED06351640815E2FF0A42
:1017700003E162515D0810E263516F080DE303E17C
:101780006251EA0809E39A0E616F990E606F110EBB
:101790005F6E820E5E6E06D0616B606B200E5F6EB8
:1017A000820E5E6ED89261C067F060C066F05FC066
:1017B00065F05EC064F0170E6B6FB70E6A6F510E66
:1017C000696F710E686F0AEC04F003C061F002C02B
:1017D00060F001C05FF000C05EF05EC000F05FC06E
:1017E00001F060C002F061C003F01200EACF5AF0CD
:1017F000E9CF59F053AE08D0598E59A8592A521E34
:10180000531E522AD8B4532A5338F009556E552620
:10181000E20F566E320F586E53500F0B5626562657
:101820005826E90F576E5726572652380F0B572662
:10183000582657365836581E583652500F0B5826D1
:101840005536070E546E0A0E57065826FDE3560607
:101850005726FDE355065626FDE354065526FDE3BF
:10186000EA6A540EE96E070E5914599CED52591448
:1018700007E159B8EE5259B803D0200E006E20D0BF
:10188000E926000EEA22E950580803E1EA5201E194
:10189000598CEF50006E08E159BC06D059B81CD0E5
:1018A00059B602D0200E0BD059AE06D02D0E006EC8
:1018B000ED50599C599E04D059865998300E0026F7
:1018C000EACF53F0E9CF52F000C063F010EC07F01C
:1018D00053C0EAFF52C0E9FFEE5059ACD4D7120012
:1018E0004BC055F04AC054F049C053F048C052F0C4
:1018F000596A586A576A7F0E566E3BEC07F0D8A0BB
:10190000E5D04BC067F04AC066F049C065F048C0FA
:1019100064F06B6B6A6B200E696F820E686F91ECDE
:1019200003F003C055F002C054F001C053F000C0F2
:1019300052F003C059F002C058F001C057F000C087
:1019400056F0CCDC03C04FF002C04EF001C04DF0A9
:1019500000C04CF04FC055F04EC054F04DC053F095
:101960004CC052F0596A586A576A7F0E566E3BEC6B
:1019700007F029E34FC067F04EC066F04DC065F038
:101980004CC064F0CD0E6B6FCC0E6A6F4C0E696F5D
:101990007B0E686F91EC03F003C055F002C054F069
:1019A00001C053F000C052F0040EE96E03C059F0BC
:1019B00002C058F001C057F000C056F0030E5A6E36
:1019C000DDEC07F081D0330E556E546E730E536EFE
:1019D0007E0E526E4FC059F04EC058F04DC057F0B9
:1019E0004CC056F03BEC07F019E34FC055F04EC029
:1019F00054F04DC053F04CC052F0660E596E586E04
:101A0000060E576E7F0E566E3BEC07F007E3460E50
:101A1000F66E000EF76E2BEC07F056D0660E556E84
:101A2000546E060E536E7F0E526E4FC059F04EC06C
:101A300058F04DC057F04CC056F03BEC07F03EE379
:101A40004FC055F04EC054F04DC053F04CC052F052
:101A5000596A586A180E576E820E566E3BEC07F0A4
:101A60002DE34FC067F04EC066F04DC065F04CC02E
:101A700064F0CD0E6B6FCC0E6A6F4C0E696F7B0EEF
:101A8000686F91EC03F003C055F002C054F001C040
:101A900053F000C052F0030EE96E03C059F002C0CB
:101AA00058F001C057F000C056F0020E5A6EDDEC3F
:101AB00007F0200E636F10EC07F006D04C0EF66EA8
:101AC000000EF76E2BEC07F0C0EF12F04BC055F094
:101AD0004AC054F049C053F048C052F0596A586A9D
:101AE000200E576E820E566E3BEC07F0D8A09ED0AB
:101AF0004BC059F04AC058F049C057F048C056F0A2
:101B00006EEC09F003C04FF002C04EF001C04DF082
:101B100000C04CF04FC055F04EC054F04DC053F0D3
:101B20004CC052F0596A586A576A7F0E566E3BECA9
:101B300007F013E3030EE96E4FC059F04EC058F0A2
:101B40004DC057F04CC056F0020E5A6EDDEC07F057
:101B5000200E636F10EC07F067D0330E556E546E95
:101B6000730E536E7E0E526E4FC059F04EC058F039
:101B70004DC057F04CC056F03BEC07F019E34FC096
:101B800055F04EC054F04DC053F04CC052F0660EAC
:101B9000596E586E060E576E7F0E566E3BEC07F070
:101BA00007E3520EF66E000EF76E2BEC07F03CD0FA
:101BB000660E556E546E060E536E7F0E526E4FC0FB
:101BC00059F04EC058F04DC057F04CC056F03BECA9
:101BD00007F024E34FC055F04EC054F04DC053F011
:101BE0004CC052F0596A586A180E576E820E566EE3
:101BF0003BEC07F013E3030EE96E4FC059F04EC003
:101C000058F04DC057F04CC056F0010E5A6EDDEC46
:101C100007F0200E636F10EC07F006D0580EF66E3A
:101C2000000EF76E2BEC07F0C0EF12F04BC055F032
:101C30004AC054F049C053F048C052F0596A586A3B
:101C4000480E576E850E566E3BEC07F0D8A0C1D0FB
:101C50004BC05BF04AC05AF049C059F048C058F038
:101C60005F6A5E6A200E5D6E820E5C6E3FEC05F070
:101C700003C055F002C054F001C053F000C052F050
:101C800003C059F002C058F001C057F000C056F030
:101C90006EEC09F003C04FF002C04EF001C04DF0F1
:101CA00000C04CF04FC067F04EC066F04DC065F00C
:101CB0004CC064F06B6B6A6B200E696F820E686FAC
:101CC00091EC03F003C067F002C066F001C065F05C
:101CD00000C064F052EC09F002C051F001C050F0B5
:101CE0004FC055F04EC054F04DC053F04CC052F0B0
:101CF000596A586A576A7F0E566E3BEC07F007E345
:101D00005E0EF66E000EF76E2BEC07F060D0330E11
:101D1000556E546E730E536E7E0E526E4FC059F058
:101D20004EC058F04DC057F04CC056F03BEC07F099
:101D300019E34FC055F04EC054F04DC053F04CC0A5
:101D400052F0660E596E586E060E576E7F0E566E26
:101D50003BEC07F007E3640EF66E000EF76E2BEC1B
:101D600007F035D04FC055F04EC054F04DC053F081
:101D70004CC052F0596A586A200E576E820E566E49
:101D80003BEC07F01EE3660E556E546E060E536E66
:101D90007F0E526E4FC059F04EC058F04DC057F0F4
:101DA0004CC056F03BEC07F00CE3020EE96E51C05C
:101DB00053F050C052F01ADD200E636F10EC07F0A4
:101DC00006D06A0EF66E000EF76E2BEC07F0C0EF31
:101DD00012F04BC055F04AC054F049C053F048C00F
:101DE00052F0596A586A7A0E576E880E566E3BEC5E
:101DF00007F0D8A0C5D04BC05BF04AC05AF049C02C
:101E000059F048C058F05F6A5E6A480E5D6E850EF4
:101E10005C6E3FEC05F003C055F002C054F001C009
:101E200053F000C052F003C059F002C058F001C096
:101E300057F000C056F06EEC09F003C04FF002C03E
:101E40004EF001C04DF000C04CF04FC067F04EC0E6
:101E500066F04DC065F04CC064F06B6B6A6B480E69
:101E6000696F850E686F91EC03F003C067F002C0E4
:101E700066F001C065F000C064F052EC09F002C0E9
:101E800051F001C050F04FC055F04EC054F04DC05D
:101E900053F04CC052F0596A586A576A7F0E566E1A
:101EA0003BEC07F00CE3020EE96E51C053F050C05A
:101EB00052F09CDC200E636F10EC07F060D04FC036
:101EC00055F04EC054F04DC053F04CC052F0660E69
:101ED000596E586E060E576E7F0E566E3BEC07F02D
:101EE00019E3330E556E546E730E536E7E0E526EA2
:101EF0004FC059F04EC058F04DC057F04CC056F08E
:101F00003BEC07F007E3700EF66E000EF76E2BEC5D
:101F100007F035D04FC055F04EC054F04DC053F0CF
:101F20004CC052F0596A586A200E576E820E566E97
:101F30003BEC07F01EE3660E556E546E060E536EB4
:101F40007F0E526E4FC059F04EC058F04DC057F042
:101F50004CC056F03BEC07F00CE3020EE96E51C0AA
:101F600053F050C052F042DC200E636F10EC07F0CB
:101F700006D0760EF66E000EF76E2BEC07F000D34F
:101F80004BC055F04AC054F049C053F048C052F01D
:101F9000596A400E586E1C0E576E8C0E566E3BECF6
:101FA00007F0D8A0A9D04BC05BF04AC05AF049C096
:101FB00059F048C058F05F6A5E6A7A0E5D6E880E0E
:101FC0005C6E3FEC05F003C055F002C054F001C058
:101FD00053F000C052F003C059F002C058F001C0E5
:101FE00057F000C056F06EEC09F003C04FF002C08D
:101FF0004EF001C04DF000C04CF04FC055F04EC047
:1020000054F04DC053F04CC052F0596A586A576AA8
:102010007F0E566E3BEC07F007E37C0EF66E000E6B
:10202000F76E2BEC07F067D04FC055F04EC054F060
:102030004DC053F04CC052F0660E596E586E060EED
:10204000576E7F0E566E3BEC07F019E3330E556E5C
:10205000546E730E536E7E0E526E4FC059F04EC0CA
:1020600058F04DC057F04CC056F03BEC07F007E37A
:10207000820EF66E000EF76E2BEC07F03CD0660E6B
:10208000556E546E060E536E7F0E526E4FC059F051
:102090004EC058F04DC057F04CC056F03BEC07F026
:1020A00024E34FC055F04EC054F04DC053F04CC027
:1020B00052F0596A586A200E576E820E566E3BECEB
:1020C00007F013E3030EE96E4FC059F04EC058F00D
:1020D0004DC057F04CC056F0010E5A6EDDEC07F0C3
:1020E0006B0E636F10EC07F006D0880EF66E000ED4
:1020F000F76E2BEC07F044D24BC055F04AC054F0B9
:1021000049C053F048C052F0596A500E586E430E01
:10211000576E8F0E566E3BEC07F0D8A098D04BC090
:102120005BF04AC05AF049C059F048C058F05F6AA5
:10213000400E5E6E1C0E5D6E8C0E5C6E3FEC05F00C
:1021400003C055F002C054F001C053F000C052F07B
:1021500003C059F002C058F001C057F000C056F05B
:102160006EEC09F003C04FF002C04EF001C04DF01C
:1021700000C04CF04FC067F04EC066F04DC065F037
:102180004CC064F06B6B6A6B200E696F820E686FD7
:1021900091EC03F003C067F002C066F001C065F087
:1021A00000C064F052EC09F002C051F001C050F0E0
:1021B0004FC055F04EC054F04DC053F04CC052F0DB
:1021C000596A586A576A7F0E566E3BEC07F007E370
:1021D0008E0EF66E000EF76E2BEC07F037D04FC068
:1021E00055F04EC054F04DC053F04CC052F0660E46
:1021F000596E586E060E576E7F0E566E3BEC07F00A
:1022000019E3330E556E546E730E536E7E0E526E7E
:102210004FC059F04EC058F04DC057F04CC056F06A
:102220003BEC07F007E3940EF66E000EF76E2BEC16
:1022300007F00CD0020EE96E51C053F050C052F0BE
:10224000F6EC0BF06B0E636F10EC07F099D14BC0FE
:1022500055F04AC054F049C053F048C052F0596A92
:10226000240E586E740E576E920E566E3BEC07F0AD
:10227000D8A0C2D04BC05BF04AC05AF049C059F058
:1022800048C058F05F6A500E5E6E430E5D6E8F0E52
:102290005C6E3FEC05F003C055F002C054F001C085
:1022A00053F000C052F003C059F002C058F001C012
:1022B00057F000C056F06EEC09F003C04FF002C0BA
:1022C0004EF001C04DF000C04CF04FC067F04EC062
:1022D00066F04DC065F04CC064F06B6B6A6B480EE5
:1022E000696F850E686F91EC03F003C067F002C060
:1022F00066F001C065F000C064F052EC09F002C065
:1023000051F001C050F04FC055F04EC054F04DC0D8
:1023100053F04CC052F0596A586A576A7F0E566E95
:102320003BEC07F007E39A0EF66E000EF76E2BEC0F
:1023300007F061D0330E556E546E730E536E7E0EE1
:10234000526E4FC059F04EC058F04DC057F04CC0BF
:1023500056F03BEC07F019E34FC055F04EC054F077
:102360004DC053F04CC052F0660E596E586E060EBA
:10237000576E7F0E566E3BEC07F007E3A00EF66E2D
:10238000000EF76E2BEC07F036D0660E556E546ECD
:10239000060E536E7F0E526E4FC059F04EC058F06D
:1023A0004DC057F04CC056F03BEC07F01EE34FC059
:1023B00055F04EC054F04DC053F04CC052F0596A25
:1023C000586A200E576E820E566E3BEC07F00DE3F6
:1023D000020EE96E51C053F050C052F0F6EC0BF013
:1023E0006B0E636F10EC07F006D0A60EF66E000EB3
:1023F000F76E2BEC07F0C4D04BC055F04AC054F038
:1024000049C053F048C052F0800E596E960E586E77
:10241000180E576E960E566E3BEC07F0D8A0AAD059
:102420004BC05BF04AC05AF049C059F048C058F060
:102430005F6A240E5E6E740E5D6E920E5C6E3FECF3
:1024400005F003C055F002C054F001C053F000C0C5
:1024500052F003C059F002C058F001C057F000C05C
:1024600056F06EEC09F003C04FF002C04EF001C010
:102470004DF000C04CF04FC055F04EC054F04DC070
:1024800053F04CC052F0596A586A576A7F0E566E24
:102490003BEC07F007E3AC0EF66E000EF76E2BEC8C
:1024A00007F067D04FC055F04EC054F04DC053F008
:1024B0004CC052F0660E596E586E060E576E7F0E67
:1024C000566E3BEC07F019E3330E556E546E730EE7
:1024D000536E7E0E526E4FC059F04EC058F04DC034
:1024E00057F04CC056F03BEC07F007E3B20EF66E27
:1024F000000EF76E2BEC07F03CD04FC055F04EC0ED
:1025000054F04DC053F04CC052F0596A586A200E36
:10251000576E820E566E3BEC07F025E3660E556E45
:10252000546E060E536E7F0E526E4FC059F04EC061
:1025300058F04DC057F04CC056F03BEC07F013E399
:10254000030EE96E4FC059F04EC058F04DC057F021
:102550004CC056F0010E5A6EDDEC07F04D0E636F65
:1025600010EC07F006D0B80EF66E000EF76E2BECEE
:1025700007F006D0BE0EF66E000EF76E2BEC07F0DD
:1025800027EF13F0F86AD09E600ED36E400E9B6E5C
:10259000646A356A346A0F015C51800B5C6F000E0F
:1025A0005D6FC196C198C19A5E6B5F6B600ED36E12
:1025B000400E9B6E646AFF0E926E936E946E640E74
:1025C000486E000177EC00F08AEF00F0640E486E70
:1025D00077EC00F0010E546EE0EC00F032EF01F009
:1025E00095EF01F014EF02F0ECEF05F003C043F0BB
:1025F00002C042F001C041F000C040F0486A496AA0
:10260000F6EC06F0DC0EF66E000EF76E2BEC07F023
:1026100043C04BF042C04AF041C049F040C048F0CE
:10262000A9EF08F0486A010E496EF6EC06F0E20EDA
:10263000F66E000EF76E2BEC07F043C04BF042C075
:102640004AF041C049F040C048F070EF0CF0E80E8D
:0E265000F66E000EF76E2BEC07F0C4D70300F9
:020000040030CA
:0E00000015C8787C000991000FC00FE00F407A
:00000001FF
